:0200000480007A
:100000006F00C0006F20802C6F20402C93000000F8
:10001000130100009301000013020000930200008E
:100020001303000093030000130400009304000076
:10003000130500009305000013060000930600005E
:100040001307000093070000130800009308000046
:100050001309000093090000130A0000930A00002E
:10006000130B0000930B0000130C0000930C000016
:10007000130D0000930D0000130E0000930E0000FE
:10008000130F0000930F000097020000938202F804
:100090007390523017A100001301C1E4F32240F124
:1000A0009392C2003301510073100134EF20900B82
:1000B000173500001305858B6F20006B8332851088
:1000C000739012148330850003310501833185015B
:1000D000033205028332850203330503833385032C
:1000E000033405048334850483358505033605060A
:1000F00083368506033705078337850703380508E8
:10010000833885080339050983398509033A050AC7
:10011000833A850A033B050B833B850B033C050CA7
:10012000833C850C033D050D833D850D033E050E87
:10013000833E850E033F050F833F850F033505057D
:10014000730020107311011423341100233C31007B
:10015000233041022334510223386102233C7102CF
:1001600023308104233491042338A104233CB104B7
:100170002330C1062334D1062338E106233CF1069F
:10018000233001092334110923382109233C310983
:100190002330410B2334510B2338610B233C710B6B
:1001A0002330810D2334910D2338A10D233CB10D53
:1001B0002330C10F2334D10F2338E10F233CF10F3B
:1001C000F312011423385100F32200102330511090
:1001D000F322101423345110F32230142338511019
:1001E000F3222014233C5110130501006F208033AB
:1010000000000000000000000000000000000000E0
:1010100000000000000000000000000000000000D0
:1010200000000000000000000000000000000000C0
:1010300000000000000000000000000000000000B0
:081040000000000000000000A8
:10200000B367B500B3E7C70093F77700B306C50021
:10201000638407023386C50093070500637ED502FB
:1020200003C705009385150093871700A38FE7FE6C
:10203000E398C5FE67800000E37ED5FE93070500A8
:1020400003B70500938787009385850023BCE7FECF
:10205000E3E8D7FE6780000067800000130101FFFE
:10206000B367C500233081002334110093F7770054
:10207000130405003307C500638207026376E50099
:1020800093F5F50FEFF09FFD8330810013050400F9
:1020900003340100130101016780000093F5F50F7F
:1020A00093968500B3E6B60093970601B3E7D70091
:1020B00093960702B3E6F600E378E5FC9307050084
:1020C0009387870023BCD7FEE3ECE7FE83308100D3
:1020D00013050400033401001301010167800000AF
:1020E00083470500638E07009307050003C71700A9
:1020F00093871700E31C07FE3385A7406780000025
:1021000013050000678000008347050093851500D4
:102110001305150003C7F5FF638A0700E386E7FE92
:102120001B8507003B05E5406780000013050000A4
:102130006FF05FFFB367B50093F77700639E070208
:10214000137886FF330805016378050393070500BC
:102150006F000001938787009385850063F807016E
:1021600083B6070003B70500E386E6FE3385A74084
:102170003306A640138507003386C5006F00400173
:1021800003C705008347F5FF93851500639AE700B1
:1021900013051500E396C5FE1305000067800000D7
:1021A0003B85E740678000009307050003C70500F3
:1021B0009387170093851500A38FE7FEE31807FEAA
:1021C000678000000347050093060002930705009F
:1021D0006318D70003C7170093871700E30CD7FED7
:1021E0009306D0026300D7069306B0026300D704BB
:1021F00083C60700930500006382060413050000F0
:1022000093871700131725001B8606FD83C607005A
:102210003307A700131717003305E600E39206FE05
:10222000638005023305A0406780000083C6170065
:102230009305000093871700E39206FC1305000046
:102240006780000083C6170093051000938717006E
:10225000E39606FA130500006FF09FFE8347050022
:10226000638007049305101017F7FFFF130787D942
:10227000939505030336070013051500B3E6B70071
:10228000630A060097F7FFFF23BE07DA83370700CC
:10229000E39A07FE2330D70083470500E39C07FC41
:1022A0006780000017F7FFFF1307C7D583370700C4
:1022B000638A070097F7FFFF23B607D88337070025
:1022C000E39A07FE2330A7006F000000130101FF0F
:1022D0001305903423341100EFF0DFFC130101FEED
:1022E0001306810093077101130890006F008000AE
:1022F000930707009376F500138706009305000304
:102300006374D800930570053B07B7002380E7008E
:10231000135545001387F7FFE31CF6FC8347810044
:10232000230C0100638207041305101093060600B6
:1023300017F7FFFF130707CD1315050383350700B4
:102340009386160033E6A700638A050097F7FFFF20
:1023500023BA07CE83370700E39A07FE83C7060038
:102360002330C700E39C07FC1301010267800000D3
:10237000130101FF37F8FFFF233411003307050174
:10238000B7E703006378F7141357C5009306076097
:1023900017360000130606C793973600B307F600FA
:1023A00083B70700337505016390070E977500002A
:1023B0009385C5C503B805006302081483378800F8
:1023C0009778000083B808C423B0F500638E170F18
:1023D0008337080093983600B308160193D7C700D7
:1023E0009397A70013E3F70D93E5F70123B0680077
:1023F00073000512972700009387C7C01317470083
:10240000B387E70003B7070063140710033708001A
:10241000B708040023B0E7000337880023B4E700BF
:10242000F3A80810B707E0FFB307F500371800005E
:10243000130705003388070103BF070083BE870029
:1024400003BE070103B387012330E7012334D7011B
:102450002338C701233C670093870702130707024D
:10246000E39C07FD7390081093973600B306F600BF
:1024700023B0B600730005120F10000083308100F6
:10248000130101016780000013F70704630A0702C4
:1024900013F70708631A07041307F00093E7070808
:1024A0006394E50493963600B306D60023B0F60095
:1024B0007300051283308100130101016780000061
:1024C00093E707046FF01FFE9777000023BC07B265
:1024D0006FF01FF0171500001305C587EFF01FD828
:1024E00013053000EFF01FDC171500001305058BF6
:1024F000EFF0DFD613053000EFF0DFDA171500003C
:102500001305458EEFF09FD513053000EFF09FD9EE
:10251000171500001305858EEFF05FD4130530000A
:10252000EFF05FD883358511130101F82338810658
:10253000233C11062334910623302107233C310527
:10254000233841052334510523306105233C7103B1
:1025500023388103233491032330A103233CB101A9
:102560009307800013040500638AF50E930720008B
:102570006380F506938745FF130710006376F70025
:102580009307F0006392F51A03350411EFF05FDE54
:102590001305040003340107833081078334810667
:1025A0000339010683398105033A0105833A810421
:1025B000033B0104833B8103033C0103833C810211
:1025C000033D0102833D8101130101086FD01FAF5C
:1025D000033785109377370063980706EF0780006D
:1025E000731030000327070083A70700630AF7046E
:1025F00013051010930710049716000093860684A5
:1026000017F7FFFF130707A013150503833507000E
:102610009386160033E6A700638A050097F7FFFF4D
:1026200023B207A283370700E39A07FE83C7060099
:102630002330C700E39C07FC13053000EFF09FC672
:1026400013051000EFF01FC61715000013050589CC
:10265000EFF0DFC013053000EFF0DFC403290505FC
:10266000371C0000972400009384C499973B000016
:10267000938B4B99370B0400B70AE0FF977D00005E
:10268000938D4D98177A0000130A4A98B7F9030002
:102690006F0080012334F70023B0FD00B71700005E
:1026A000330CFC00630E3C0B9357CC001394470093
:1026B0003387840003370700E30207FE9387076030
:1026C00093973700B387FB0083BC070093F70C0494
:1026D000638E0706732D0B1037160000B3055C01DF
:1026E00013050C002334B100EFF0DFA4630E0500E6
:1026F00093FC0C088335810063800C0437160000BE
:1027000013050C00EFF0DF8FB387840073100D10FA
:1027100003B70D0023B00700E31E07F623B0FD004A
:102720002330FA006FF09FF7170500001305857D31
:10273000EFF0DFB26FF05FF017050000130585764C
:10274000EFF0DFB113053000EFF0DFB51705000043
:102750001305C571EFF09FB013053000EFF09FB483
:1027600013050900EFF01FB4F32740F1639A07182F
:102770009757000093870789130101ED93D7C7008E
:1027800023308112176800001308C887130405005E
:102790009397A700174500001305C586233411122F
:1027A0009356C5001357C80093E7170097380000E9
:1027B000938848851306F0FF233CF5FE9396A60008
:1027C0001317A700B707002093E61600136717003A
:1027D00093D5C8001313F6039387F70C233CF8FE38
:1027E00023B0D8002330E500B3E7650073900718E5
:1027F00073270018639EE7141356B6009307F00181
:102800009702000093824201F39252307310063B0C
:102810007390073A739052301308F0BF13185801A1
:1028200097E7FFFF93874792B3870701739057108D
:10283000F3270034B387070173900714B7B700007C
:102840009B87071073902730B7E701009B870760CD
:10285000739007307350403017270000130787B973
:102860009307083EB3060701B307F700B70808004F
:1028700017660000233CD67817230000130383F665
:102880009766000023B0F6789388F8039307D00288
:102890001308080113D61700B3861701B347F600D3
:1028A000B30507019396C600939757002330D700CE
:1028B0002334B70093F7070213070701B367F60045
:1028C000E31AE3FC13060012930500001305010050
:1028D0009727000023B407F0EFF04FF8B707008008
:1028E0003304F4001305010023348110EFD00FFDF1
:1028F0008330811203340112130101136780000039
:1029000013071000B717540537060800938757B20E
:102910001306C6FF1315F7019316E7036F00C001F6
:102920002F20070013D71700B3C7E7009397E703DB
:10293000B3F7D700B3E7E70033F7C70093F5170005
:102940003307A700E39E05FC032007006FF09FFDFF
:10295000170500001305055EEFF05F9013053000CA
:10296000EFF05F946780000097000000938080691B
:1029700003B70000B703FF009B83F30F939303019A
:102980009383F30F939303019383F30F9301200039
:102990006312773A970000009380C06603B7800007
:1029A000B70301FF9B8313F093930301938313F009
:1029B00093930301938303F093013000631C7736F4
:1029C000970000009380006403B70001B703010083
:1029D0009B8313F093930301938313F09393030169
:1029E000938313F09393C300938303FF93014000F9
:1029F00063127734970000009380C06003B78001B2
:102A0000B703FFFF9B83F30F939303019383F30FAC
:102A1000939303019383F30F9393C3009383F30082
:102A20009301500063187730970000009380005F97
:102A300003B780FEB703FF009B83F30F939303015B
:102A40009383F30F939303019383F30F9301600038
:102A50006312772E970000009380405C03B700FF5D
:102A6000B70301FF9B8313F093930301938313F048
:102A700093930301938303F093017000631C772AFF
:102A8000970000009380805903B780FFB7030100CF
:102A90009B8313F093930301938313F093930301A8
:102AA000938313F09393C300938303FF93018000F8
:102AB00063127728970000009380405603B7000008
:102AC000B703FFFF9B83F30F939303019383F30FEC
:102AD000939303019383F30F9393C3009383F300C2
:102AE0009301900063187724970000009380805131
:102AF000938000FE83B20002B703FF009B83F30FB5
:102B0000939303019383F30F939303019383F30F41
:102B10009301A00063907222970000009380804E82
:102B20009380D0FF83B2B000B70301FF9B8313F003
:102B300093930301938313F093930301938303F01F
:102B40009301B0006398721E9301C000130200004D
:102B5000970000009380804B03B7800013030700A9
:102B6000B70301009B8313F093930301938313F046
:102B700093930301938313F09393C300938303FF11
:102B8000631A731A1302120093022000E31252FC1C
:102B90009301D0001302000097000000938080474B
:102BA00003B780001300000013030700B703FFFF03
:102BB0009B83F30F939303019383F30F9393030189
:102BC0009383F30F9393C3009383F30063147316FB
:102BD0001302120093022000E31052FC9301E00064
:102BE00013020000970000009380C04103B78000EB
:102BF000130000001300000013030700B70301FFD8
:102C00009B8313F093930301938313F09393030136
:102C1000938303F0631073121302120093022000D7
:102C2000E31252FC9301F000130200009700000031
:102C30009380C03D03B78000B70301009B8313F06E
:102C400093930301938313F093930301938313F0FE
:102C50009393C300938303FF631E770C1302120048
:102C600093022000E31452FC9301000113020000C0
:102C7000970000009380003A1300000003B7800023
:102C8000B703FFFF9B83F30F939303019383F30F2A
:102C9000939303019383F30F9393C3009383F30000
:102CA000631A77081302120093022000E31252FC09
:102CB00093011001130200009700000093808034FC
:102CC000130000001300000003B78000B70301FFEA
:102CD0009B8313F093930301938313F09393030166
:102CE000938303F063187704130212009302200009
:102CF000E31452FC970200009382C23003B1020039
:102D0000130120009303200093012001631471023A
:102D1000970200009382022F03B10200130000000B
:102D2000130120009303200093013001631471000C
:102D3000631A300013951100630005001365150038
:102D4000730000001305100073000000731000C032
:102D5000417373657274696F6E206661696C656436
:102D60003A2061646472203E3D202831554C203C5D
:102D70003C203132292026262061646472203C20C8
:102D80003633202A202831554C203C3C2031322932
:102D90000A00000000000000417373657274696FDF
:102DA0006E206661696C65643A20212870745B331B
:102DB0005D5B616464722F2831554C203C3C2031AE
:102DC00032295D20262030783038302920262620F0
:102DD0006361757365203D3D203078660A00000010
:102DE000417373657274696F6E206661696C6564A6
:102DF0003A206E6F64650A00417373657274696F7F
:102E00006E206661696C65643A20757365725F6DEA
:102E1000617070696E675B616464722F2831554C14
:102E2000203C3C203132295D2E61646472203D3D9E
:102E300020300A0000000000417373657274696FEE
:102E40006E206661696C65643A202122696C6C654C
:102E500067616C20696E737472756374696F6E223A
:102E60000A00000000000000417373657274696F0E
:102E70006E206661696C65643A2070745B335D5BDB
:102E8000616464722F2831554C203C3C203132293A
:102E90005D20262030783034300A00000000000029
:102EA000417373657274696F6E206661696C6564E5
:102EB0003A2070745B335D5B616464722F28315516
:102EC0004C203C3C203132295D202620307830389F
:102ED000300A000000000000417373657274696F6E
:102EE0006E206661696C65643A2074662D3E65707B
:102EF0006320252034203D3D20300A0000000000E2
:102F0000417373657274696F6E206661696C656484
:102F10003A202122756E657870656374656420655A
:102F20007863657074696F6E220A0000000000000B
:102F3000417373657274696F6E206661696C656454
:102F40003A202122756E737570706F7274656420FB
:0C2F500073617470206D6F6465220A00CC
:10300000FF00FF00FF00FF0000FF00FF00FF00FFC8
:10301000F00FF00FF00FF00F0FF00FF00FF00FF0B8
:040000058000000077
:00000001FF
